:020000040000FA
:100000000A20003086008500FF3087001328031384
:1000100083120800031383160800031783120800D5
:1000200003178316080064204A203B20322000304A
:100030009500212052203B203220013095002120C4
:1000400014280D20103093073E2094000030072024
:1000500086000D201508072085000D2014080720B4
:10006000860008003E2014081002031D38283A2894
:10007000930A322808000030930008000D2013086E
:100080008D0010208C130C140C1844280D200C0823
:1000900094000800072007080D209100110E0F3969
:1000A000900008000D2000309200072007080D2066
:1000B0009400141892159418121514199214941986
:1000C00012141208900008000D20053093003E2005
:1000D00005301402031D73281E3093003E20673044
:1000E00014020319152900308D0000308C001621F0
:1000F00001308D0001308C00162102308D0002305D
:100100008C00162103308D0003308C001621043042
:100110008D0004308C00162105308D0005308C00D8
:10012000162106308D0006308C00162107308D0018
:1001300007308C00162108308D0008308C00162105
:1001400009308D0009308C0016210A308D000A30EC
:100150008C0016210B308D000B308C0016210C30DA
:100160008D000C308C0016210D308D000D308C0070
:1001700016210E308D000E308C0016210F308D00B0
:100180000F308C00162110308D00FC308C001621B1
:1001900011308D0060308C00162112308D00DA3065
:1001A0008C00162113308D00F2308C001621143093
:1001B0008D0066308C00162115308D00B6308C0015
:1001C000162116308D00BE308C00162117308D00A0
:1001D000E0308C00162118308D00FE308C00162186
:1001E00019308D00F6308C0016211A308D00FD304C
:1001F0008C0016211B308D0061308C0016211C30C4
:100200008D00DB308C0016211D308D00F3308C000A
:1002100016211E308D0067308C0016211F308D0096
:10022000B7308C00162110200C11080010200C157E
:1002300055308D00AA308D008C148C181D290C129D
:040240000D20080085
:02400E00F13F80
:00000001FF
